:0600000018308A00002FF9
:08000800FF00030E8312FE004D
:100010000A08FA008A018C1E26280408FC003C0805
:1000200084001A08243A031D17283F1522281A08AD
:1000300080000008BC0A3C1A3C120D3A2011031D36
:10004000242820154030BC007C0884007A088A00EF
:0A0050007E0E8300FF0E7F0E0900F4
:100080008A150A160A2F8A150A160B2F4928C02925
:100090002C2C210E07398207BF2CBF2C002B002BE4
:1000A000352B352B942821080F39820766289D2C83
:1000B000A02CA92CA32CA62C352B762D862D862D95
:1000C000A12DA72D8C2DAC2DB62DC72D22083F3983
:1000D0008207442B3A2BBD29462BC329482B4A2B98
:1000E000072BD42C2E2DD02B4C2BBD2CCB2C2F2CD6
:1000F000662C7A2C7A2C7A2C7A2C8A2C892C742CCB
:100100006E2C772C712CC52CC82C822D7B2DCF2CDE
:100110005F2CB229CC2D8207013402340434083418
:100120001034203440348034210803398207822C73
:100130007D2C352B22080F398207D52DD82DDB2DAC
:10014000DE2D352B352B3F2BD02DE12DE62D352BFC
:10015000352B352B352B352B352B6430BE00B22893
:100160000A30BE00C020BE0BB22808000530C128EE
:100170000230C1280030C1280330C1280430C12812
:10018000063083168100831281016400473001022A
:10019000031CC52800308316810083120034FB2124
:1001A000AE001530AD002D08073A0319DF28CF3017
:1001B0002E020318DF280530AE07AD03D328063022
:1001C00095002D08831692008312B028950108002F
:1001D0007B13CF208316813087008312871107128B
:1001E00087102321B801B90187166B21B02087122F
:1001F0008714B0205121871087166B21B0208712F9
:100200008714FB21AD00B0200122AE002321A01DE8
:100210001121871087166B21B0208712871423299C
:10022000003448212A212A212A212A212A212A216F
:100230002A2151213F30A1057F30A2053C21932185
:10024000B801B90108008101640027300102031CD4
:1002500024290034B90A0319B80A0630AF00063061
:10026000A5002F1C07122F18071687150F228711BC
:10027000AF0CA50B3129003421083F39B00022080A
:10028000B100BF10211BBF140230A0190330211B85
:1002900000302E214C2171213008A1003108A2002C
:1002A00000340430A01905302E218711071683165B
:1002B00007168312A101A2011030A50087150310B3
:1002C000A10CA20C071AA1178711A50B5E29031018
:1002D000A10CA20C211364008316071283120712CB
:1002E00000340310A20DA10D1030A50087152218AF
:1002F0000716221C0712A10CA20C8711A50B762948
:10030000003408302E21B620B620080083161208CB
:100310008312B500BE201130350203180800BE203C
:10032000B50A8B290800201364000230A01903309D
:100330002E214C21712181210430A01905302E215C
:100340002321552131082206031DAC29A01951296A
:1003500030082106031951290E30A100EE30A20009
:1003600020170034E820AD2048212A212A212A2103
:100370002A212A212A215121302B51212A21352BB2
:100380003C21BF18352B93212A21352BBD003D0E72
:10039000CA213D080F393038AF00393C0318D22943
:1003A0000730AF072F08AF006430B7003F19DD29D1
:1003B000B60BE029B70BE029000000008616080004
:1003C0006400061AD6292F0899002321831698184D
:1003D000E729981CE92983128612B7013F19DD2904
:1003E000061EF42986160800BE0BEE296400B70B22
:1003F000EE2986160800C130022AD130022AE130E7
:10040000022AC9309F000F221F150F221F19062A2A
:1004100023211F150F221F190B2A0F221E0864000B
:100420000800C0303A04F5003B08F6002012A50190
:10043000071E272A87156400071E272AA60B1B2ADA
:10044000A50B1B2A20168316071683120800E0301E
:10045000F1005F225F225F225F22A501F701871171
:100460005F22A0108715071A382AA50B332A222AE3
:10047000A501A60B3F2A6400A50B3F2A222AF70AF2
:100480000319A014071A392A87115F2287157422CD
:10049000F113F51BF1170310071A0314F60DF50DF0
:1004A0008316071283120712F11B07168711742295
:1004B000831607168312F10A711E462A232A640046
:1004C000BF1B672AF10AF11D5F2AF11108006400C1
:1004D0000000000000000000000000000000F10A21
:1004E000711F672A711308007708A6006400BF1BFC
:1004F0007D2AA60B772AA01C0800640000000000DB
:100500000000000000000000A60B7D2AA01C0800CF
:1005100064008A2AA60B882A08007308F600623055
:10052000F50016225F227008F6006130F5001622F1
:100530005F227408F6006330F50016225F22F60091
:100540006030F50016225F2A2A2138083A06031D7A
:10055000A42A39083B06031DA42A08004030F500F0
:1005600032197514A7132713B218A71732182717B3
:100570002708F60008002208B200A701A030840076
:10058000AE2216225F22A70AAE221622760880002B
:10059000840A0408E03A031DC22A84137F30F50060
:1005A000F601162208004030201B4130F5003208C9
:1005B000F6000800831603178C13FB1A8C170C1413
:1005C0000000FF3EFF3EFF3EFF3E64008312031328
:0205D000080021
:1006000021081F39BA002208BB00A522352B0B1781
:10061000E820AD2048212A212A212A212A212A2125
:100620002A212A2151210E30A105CF30A2053C21DB
:1006300093217F30A1007F30A2003C210730A7002A
:1006400006302E21A70B202B01302E2107302E2122
:1006500008302E21862101302E2107302E21B02096
:100660007B13E6208710871623212108D321220837
:10067000D32143287B13E620871087162321831676
:10068000993087008312302BE820352B2A21352B17
:10069000A011352BA015352B8316803087008312CF
:1006A000A201A10150308400FB218000840A87123E
:1006B000C0200122AF008000840A57302F020318A7
:1006C000221413302F02031C22148716B02001229B
:1006D000AF008000840A0F302F020318A214CF202D
:1006E00087128714AD2001228000840AAF00BB303E
:1006F0002F02031822158D302F02031C221587109C
:1007000023218716BC20071000008618A2150714A5
:100710000000861CA21507100716FF21C020FF212C
:10072000AF00B0008000840A77302F02031C22162D
:100730000712FF21C020FF21AF008000840A0F3084
:100740002F020318A2168715FD21C020FD21B1003C
:10075000AF008000840A7F302F02031C221787110C
:10076000FD21C020FD21AF008000840A0D302F0242
:100770000318A2178316813087008312E62022080F
:10078000E5007B13FB17D12BE6208710871623216A
:1007900083169930870083126508A200A101352BCA
:1007A000FB13F0018316F0018312E8205121210888
:1007B000EA002208EB00E620B020E8202830A10063
:1007C0000030A2003C219321C020E620B0208711F8
:1007D00083160716871183120530B6008716B020DE
:1007E0008712B020871523218711B0201830F6001A
:1007F0006130F50016225F228030F500F6011622E6
:10080000201E042CB60BEE2BE8206A08A1006B0812
:10081000A2003C219321C020E620B020871583163A
:1008200007168312B02087108716B0208712B020D9
:100830000730B6002321071E222CB60B1A2CFB1BF7
:10084000C42B282C7B17FB1BC42B342C87155F2251
:10085000000000008711352B3F14C020342CFF30DE
:10086000F500F60116225F2220107F30F500F60118
:100870001622201A282C75081F39A3007608A40018
:100880005F22F501F60116225F221030F500F60115
:1008900016227608F2005F222030F500F6011622BB
:1008A0007608F0005F223030F500F6011622760857
:1008B000F3007F30F500F60116227608F4002308D5
:1008C000A1002408A2003F1C352B432820143F1010
:1008D0001122C020A1010130A200352B7208A20014
:1008E000352B7308A200352B7008A200352B740835
:1008F000A200352B2208F800352B2208F6006530BF
:10090000F500922C2208F6006430F50016225F22D2
:10091000352BF30A4030F5007308F600F81875140B
:100920007818F61716225F227F30F500F60116229E
:100930000030D3217608D32143282208F200352B3A
:100940002208F300352B2208F000352B2208F40092
:10095000352B22089F225030F5007308F600F81856
:1009600075147818F61716225F2272089F227F30BE
:10097000F500F60116225F22352B8D22352B21083A
:100980001F39BA002208BB00352B87108716352B7C
:1009900087108712352B871523218711352BA1014D
:1009A000A20120182214352BE8200730FB18DB2C7D
:1009B0001F307B180E30BA00E0307B1C0030BB00CB
:1009C000A52203171730FB18E82C0F307B180630D0
:1009D0008F00E0307B1C00308D000313FB167B1270
:1009E000DA2203170E080313A10003170C080313E0
:1009F000A2008A013C2193212A2103178D0A0319A1
:100A00008F0A0F080313FB1C072D083A0A2D7B18C9
:100A1000083A7B1C103A031DF02CFB1248212A21B6
:100A20002A212A212A212F30FB18192D2F307B183B
:100A30002E30A100E0307B1C0030A2003C2193212D
:100A40002A212A212A2151213730A1053F30A20530
:100A50003C2193210000302B0000352BE820A4011D
:100A60000830FB18362D10307B1C2030A30051219C
:100A70002A2121083F393F3A031D742D220A031D04
:100A8000742DA40B372DA30B372D7F30A100FF3021
:100A9000A2003C210630A40051212A2121083F391F
:100AA0003F3A031D742D220A031D742DA40B4C2DF7
:100AB0002A2151212A2121083F393F3A031D742D53
:100AC0002208FF397F3A031D742D0830A4005121FC
:100AD0002A2121083F393F3A031D742D220A031DA4
:100AE000742DA40B672D302BAC21302B22088316DC
:100AF00092008312C0200122A200831612088312E2
:100B0000A100352BFB21A200A101352B20132118B8
:100B100020172208B200352B2208A700A03084003D
:100B2000D32216225F22B20AD32216227608800030
:100B3000840AA70B922D84137F30F500F60116224C
:100B4000A22DBB220030D3213208D3214028BF136D
:100B500022080319BF17352B2208A700A0308400F4
:100B60000008D321840AA70BB02D40282208A70033
:100B7000A03084000008990083169818BD2D981C99
:100B8000BF2D83122321840AA70BBA2D40280230DF
:100B9000A1002130A200352BA1010130A200352B8C
:100BA000A101A2017B1B2214352B7B10FB10352BDE
:100BB0007B14FB10352B7B10FB14352B7B14FB14A3
:100BC000352B6808E6006908E700352BAE01AD015A
:100BD000FB1669086706031DF62D68086606031DE7
:100BE000F62D2D08A1002E08A200352B680803174A
:100BF0008F000313690803178D000313DA22031013
:100C000003170C080313AE070318AD0A03170E08E9
:0C0C10000313AD07E90A0319E80AE92DF7
:100DC000ED00030883160317F00083160408EE00F5
:100DD0000A08EF001F308A000E08EB000317831685
:100DE000E030EC0506178613831286138316EC0A8F
:100DF0006C1DF72E6C1183126400061BFC2E640020
:100E0000061FFF2E86178316EC0AEC1D042FEC112B
:100E1000831286136400061B0A2F6400061F0D2F21
:100E200003108316EC1B031483128613031C86170E
:100E3000061B182F831686176400EC0A8312031012
:100E4000861B03148316EC130318EC17831264003B
:100E5000061F272F86138316861303106B1B03149C
:100E600083128613031886176400061B342F83161B
:100E7000861703108F0DEB0DEC0A83120310861BEF
:100E80000314831603180F146C1E262FEC1F522F09
:100E90006B088E006E0884006F088A00700883005B
:100EA0006D0808006B0E073982077C2F802F7E2F7C
:100EB000822F682F742F5D2F6F2F6B0807398207E1
:100EC000842F8A2F872F8D2F902F9C2F6F2F6F2F7E
:100ED00083136B1883170F08840000088F00831298
:100EE0006400061F702FEE2E83136B1883170F08F4
:100EF00084006D0880006F2F6D086E2F6E086E2FB6
:100F000070086E2F6F086E2F0F08ED006F2F0F08FF
:100F1000EE006F2F0F08F0006F2F0F08EF006F2FFC
:100F20000F0883128C0083168C130C1555308D001E
:100F3000AA308D008C146F2F0F0883128D0083163A
:0C0F40008C130C1483120C0883166E2F07
:101E00007011031970157013031B7017F012831AE9
:101E1000F01603178316ED006430F00503089B39B4
:101E2000F0040408EE000A08EF001F308A000E08D4
:101E3000EB0003178316E030EC05061786138312B8
:101E400086138316EC0A6C1D222F6C11831264001A
:101E5000061B272F6400061F2A2F86178316EC0AFD
:101E6000EC1D2F2FEC11831286136400061B352FF7
:101E70006400061F382F03108316EC1B0314831213
:101E80008613031C8617061B432F831686176400D0
:101E9000EC0A83120310861B03148316EC13031839
:101EA000EC1783126400061F522F861383168613C5
:101EB00003106B1B03148312861303188617640028
:101EC000061B5F2F8316861703108F0DEB0DEC0A90
:101ED00083120310861B0314831603180F146C1E41
:101EE000512FEC1F842F6B088E006F088A006E083C
:101EF00084007008830083160317ED0E6D0E701FAB
:101F00000313F01E831208006B0E07398207AE2FF1
:101F1000B22FB02FB42F9A2FA62F8F2FA12F6B087F
:101F200007398207B62FBC2FB92FBF2FC22FCE2F54
:101F3000A12FA12F83136B1883170F0884000008AB
:101F40008F0083126400061FA22F192F83136B18B2
:101F500083170F0884006D088000A12F6D08A02F43
:101F60006E08A02F7008A02F6F08A02F0F08ED009B
:101F7000A12F0F08EE00A12F0F08F000A12F0F08CE
:101F8000EF00A12F0F0883128C0083168C130C1501
:101F900055308D00AA308D008C14A12F0F088312AC
:101FA0008D0083168C130C1483120C088316A02F3B
:102E00007011031970157013031B7017F012831AD9
:102E1000F01603178316BD006430F00503089B39D4
:102E2000F0040408BE000A08BF001F308A000E0824
:102E3000BB0003178316E030BC0506178613831208
:102E400086138316BC0A3C1D222F3C11831264009A
:102E5000061B272F6400061F2A2F86178316BC0A1D
:102E6000BC1D2F2FBC11831286136400061B352F47
:102E70006400061F382F03108316BC1B0314831233
:102E80008613031C8617061B432F831686176400C0
:102E9000BC0A83120310861B03148316BC13031889
:102EA000BC1783126400061F522F861383168613E5
:102EB00003103B1B03148312861303188617640048
:102EC000061B5F2F8316861703108F0DBB0DBC0AE0
:102ED00083120310861B0314831603180F143C1E61
:102EE000512FBC1F842F3B088E003F088A003E08EC
:102EF00084007008830083160317BD0E3D0E701FFB
:102F00000313F01E831208003B0E07398207AE2F11
:102F1000B22FB02FB42F9A2FA62F8F2FA12F3B089F
:102F200007398207B62FBC2FB92FBF2FC22FCE2F44
:102F3000A12FA12F83133B1883170F0884000008CB
:102F40008F0083126400061FA22F192F83133B18D2
:102F500083170F0884003D088000A12F3D08A02F93
:102F60003E08A02F7008A02F3F08A02F0F08BD001B
:102F7000A12F0F08BE00A12F0F08F000A12F0F08EE
:102F8000BF00A12F0F0883128C0083168C130C1521
:102F900055308D00AA308D008C14A12F0F0883129C
:102FA0008D0083168C130C1483120C088316A02F2B
:063BFA00020021000100A1
:103C00008101640027300102031C012E0034831659
:103C100006118312A70164008C1A1E2EBE0B0B2EF8
:103C2000A70B0B2E831606158312A70164008C1AAE
:103C30001E2EBE0B162EA70B162E072E8A110A1249
:103C4000BE208A150A168C121A08553A03193C2E02
:103C5000A01E382EA012831619080B3A0B30031938
:103C600003309900831218121816033A031D072E09
:103C7000A01618121816072E75304B268316061537
:103C800083124030BC00C0308B00352F21084B26FA
:103C900022084B26352FAF006430B7003F19552E50
:103CA000B60B582EB70B582E0000000086160800E1
:103CB0006400061A4E2E2F089900000083169818EB
:103CC0005F2E981C612E83128612B7013F19552E64
:103CD000061E6C2E86160800BE0B662E6400B70BFF
:103CE000662E86160800BF112F300002031CBF1578
:0E3CF0003A300002031C080007308002080072
:103E00000C2F8A110A1246288A110A1247288A1191
:103E10000A124828352F392FC03087002F308500EF
:103E2000FB30860095010F3097008316DF30860047
:103E3000993087003F30850003309F0020308C0090
:103E400024309800033099008101153092008312CC
:103E500012158710871690309800A001BF01FB0152
:103E6000F801BA01BB01A012072EC0308B00403010
:103E7000BC0064003F193F1118191A08981C422F02
:103E800018121816201C462F071E072F201D392F29
:103E900020113F104030840000080319840A732663
:103EA000BF19392F000EF039A100840A7326BF19FB
:103EB000392F00080F39A104840A7326BF19392F3E
:103EC000000EF039A200840A7326BF19392F0008AA
:103ED0000F39A2042108E039403A0319E62F7B1D6F
:103EE000752F2108C0390319F02F7B112108633A7F
:103EF000031D842F2208563A0319892F2208653A98
:103F0000031D842F7B15462EFB117B11A11B042F53
:103F1000012FFB15462E83160F308100831264009B
:103F2000690803178D000313680803178F00031334
:103F3000220803178C000313210803178E00831631
:103F400003178C170C158B1355308D00AA308D007C
:103F50008C140000FF3EFF3EFF3EFF3EFF3EFF3E53
:103F6000FF3EFF3EFF3EFF3EFF3EFF3EFF3EFF3E69
:103F7000FF3EFF3EFF3EFF3E0C118C1383016400A9
:103F80000D1EBF2F0D1283168101831269080317BE
:103F90008D000313680803178F00DC2783120317B3
:103FA0000C080313A20003170E080313A100080056
:103FB000E90A0319E80A0800831603178C170C1482
:103FC0000000FF3EFF3E8C138301080021081F39CB
:103FD000E8001F3A031968122208E900C627462E96
:103FE00068081E391E3A0319FC2F6808031DFB2FB1
:0C3FF0006908C039031D8B27D827462E16
:02400E002D2F54
:00000001FF
